:100000000C9434000C94D8000C943E000C943E00E8
:100010000C943E000C943E000C943E000C943E0068
:100020000C943E000C943E000C943E000C943E0058
:100030000C943E000C943E000C943E000C943E0048
:100040000C943E000C943E000C943E000C943E0038
:100050000C943E000C943E000C943E000C943E0028
:100060000C943E000C943E0011241FBECFEFD8E04C
:10007000DEBFCDBF0E94C4000C948E030C94000020
:1000800080E480937C00EAE7F0E0808180648083F4
:10009000808184FFFDCFEAE7F0E08081806180838A
:1000A0002091780030917900822F932F08954F92FC
:1000B0005F926F927F928F929F92AF92BF92CF92F8
:1000C000DF92EF92FF920F931F93DF93CF93CDB701
:1000D000DEB728970FB6F894DEBF0FBECDBF2A015A
:1000E0003B0109831A832B833C83AA2797FDA095A4
:1000F000BA2FBC01CD010E947702A30192010E9498
:1001000078016D837E838F839887C501B401A70131
:1001100096010E9478014B015C0169817A818B8193
:100120009C81A30192010E9478019B01AC01C50151
:10013000B4010E94E1019B01AC016D817E818F8140
:1001400098850E942B03A70196010E9479010E94C5
:1001500049029B01AC01862F932F28960FB6F89485
:10016000DEBF0FBECDBFCF91DF911F910F91FF90EA
:10017000EF90DF90CF90BF90AF909F908F907F9047
:100180006F905F904F90089581E084B980E48093F0
:100190007C0087E880937A00E9E6F0E08081816066
:1001A0008083EDE3F0E08081816080837894FFCFED
:1001B0001F920F920FB60F9211248F929F92AF92BF
:1001C000BF92CF92DF92EF92FF920F931F932F93E4
:1001D0003F934F935F936F937F938F939F93AF93CF
:1001E000BF93EF93FF9380E00E94400040E050E017
:1001F00060E070E000E010EC2FE734E46A017B017E
:100200000F2EF0E08F2EF0E09F2EFAE7AF2EF4E4F1
:10021000BF2EF02D0E945700E5E2F0E02081216022
:100220002083AA2797FDA095BA2FBC01CD010E947B
:1002300077025B016C0120E030E04AE753E40E9462
:100240002B037B018C0120E030E040E85FE30E945B
:10025000DD0188231CF461E070E023C0C801B70110
:1002600020E03FEF4FE757E40E9427031816ACF455
:10027000C601B50120E030E040E251E40E942B03CA
:100280000E944902CB01672B79F029E130E0F901A6
:100290003197F1F70197D9F707C0C801B7010E945C
:1002A0004902CB010197F1F7E5E2F0E080818E7F12
:1002B000808388EA91E60197F1F7FF91EF91BF9172
:1002C000AF919F918F917F916F915F914F913F91EE
:1002D0002F911F910F91FF90EF90DF90CF90BF90E3
:1002E000AF909F908F900F900FBE0F901F9018951A
:1002F0005058BB27AA270ED070C161D130F066D10B
:1003000020F031F49F3F11F41EF456C10EF4E09535
:10031000E7FB4CC1E92F72D180F3BA17620773076C
:100320008407950718F071F49EF58AC10EF4E095E4
:100330000B2EBA2FA02D0B01B90190010C01CA019F
:10034000A0011124FF27591B99F0593F50F4503E4A
:1003500068F11A16F040A22F232F342F4427585F3C
:10036000F3CF469537952795A795F0405395C9F754
:100370007EF41F16BA0B620B730B840BBAF091500C
:10038000A1F0FF0FBB1F661F771F881FC2F70EC0AB
:10039000BA0F621F731F841F48F48795779567957E
:1003A000B795F7959E3F08F0B3CF9395880F08F067
:1003B0009927EE0F979587950895D4D008F481E09A
:1003C00008950CD00AC102D140F0F9D030F021F4E8
:1003D0005F3F19F0EBC0511134C1EEC00FD198F35B
:1003E0009923C9F35523B1F3951B550BBB27AA27B6
:1003F00062177307840738F09F5F5F4F220F331F28
:10040000441FAA1FA9F333D00E2E3AF0E0E830D0F3
:1004100091505040E695001CCAF729D0FE2F27D0F6
:10042000660F771F881FBB1F261737074807AB07C4
:10043000B0E809F0BB0B802DBF01FF2793585F4F39
:100440002AF09E3F510568F0B1C0FBC05F3FECF35E
:10045000983EDCF3869577956795B795F7959F5FFE
:10046000C9F7880F911D9695879597F90895E1E052
:10047000660F771F881FBB1F621773078407BA07B1
:1004800020F0621B730B840BBA0BEE1F88F7E0950C
:100490000895BCD088F09F5790F0B92F9927B75195
:1004A000A0F0D1F0660F771F881F991F1AF0BA9538
:1004B000C9F712C0B13081F0C3D0B1E00895C0C017
:1004C000672F782F8827B85F39F0B93FCCF386952E
:1004D00077956795B395D9F73EF49095809570958B
:1004E00061957F4F8F4F9F4F0895E89409C097FB08
:1004F0003EF490958095709561957F4F8F4F9F4FFB
:100500009923A9F0F92F96E9BB279395F69587953E
:1005100077956795B795F111F8CFFAF4BB0F11F401
:1005200060FF1BC06F5F7F4F8F4F9F4F16C08823A8
:1005300011F096E911C0772321F09EE8872F762FDE
:1005400005C0662371F096E8862F70E060E02AF01F
:100550009A95660F771F881FDAF7880F969587950B
:1005600097F90895990F0008550FAA0BE0E8FEEFE0
:1005700016161706E807F907C0F012161306E40767
:10058000F50798F0621B730B840B950B39F40A2660
:1005900061F0232B242B252B21F408950A2609F43E
:1005A000A140A6958FEF811D811D089597F99F6742
:1005B00080E870E060E008959FEF80EC08950024EB
:1005C0000A941616170618060906089500240A94B8
:1005D00012161306140605060895092E0394000C3E
:1005E00011F4882352F0BB0F40F4BF2B11F460FFCD
:1005F00004C06F5F7F4F8F4F9F4F089557FD9058F6
:10060000440F551F59F05F3F71F04795880F97FBD6
:10061000991F61F09F3F79F0879508951216130690
:100620001406551FF2CF4695F1DF08C016161706BF
:100630001806991FF1CF86957105610508940895F4
:10064000E894BB2766277727CB0197F908958ADFBF
:1006500008F48FEF08950BD0C0CFB1DF28F0B6DFDC
:1006600018F0952309F0A2CFA7CF1124EACFC6DF57
:10067000A0F3959FD1F3950F50E0551F629FF001B5
:10068000729FBB27F00DB11D639FAA27F00DB11D0E
:10069000AA1F649F6627B00DA11D661F829F222797
:1006A000B00DA11D621F739FB00DA11D621F839F1E
:1006B000A00D611D221F749F3327A00D611D231FF4
:1006C000849F600D211D822F762F6A2F11249F5742
:1006D00050408AF0E1F088234AF0EE0FFF1FBB1F65
:1006E000661F771F881F91505040A9F79E3F510504
:1006F00070F05CCFA6CF5F3FECF3983EDCF38695BD
:1007000077956795B795F795E7959F5FC1F7FE2BAE
:10071000880F911D9695879597F90895F894FFCFC6
:00000001FF
